:0600000000308A006228B6
:10000800F70003088301B4000408B5000A08B60025
:100018008A017008B7007108B8007208B90073083F
:10002800BA007408BD007508BC007608BB008316CA
:0800380003130C1C2A2883129B
:100040000C1C2A28831203130C10FF308F00EF3092
:100050008E00A9208B190B1C49280B10003083122D
:100060000313861B0130A0000030061B0130A100E5
:1000700022060319472820082106031D4428A30847
:100080000319A403A3034728A30A0319A40A2108F8
:10009000A200031383123708F0003808F100390872
:1000A000F2003A08F3003D08F4003C08F5003B0874
:1000B000F6003508840036088A0034088300F70EFD
:1000C000770E09002030840034306A200C2A0406A0
:1000D0008001840A0406031D672864000034F601C9
:1000E000F401F50172087304031D7928F001F10190
:1000F00000341F30F6040310F60AF20DF30D031C52
:100100007C28F30CF20C73087102031D8928720815
:100110007002031C91287208F0027308031C730A12
:10012000F102F40DF50DF60BF61A8128F61F9D2845
:10013000F409F40A0319F503F5097408F2007508C7
:10014000F300761F0034F009F00A0319F103F109F6
:1001500000348301AA0A05302A02031C6A29AA0175
:100160006A29051701308A002508DE21A900290C1B
:10017000F000700C0139AB00290EF000F00C700C8F
:100180000139AC00290C0139AD00290EF000700CCA
:100190000139AE0029080139AF00290CF000F00C3C
:1001A000700C0139B000290E0139B100290D290D5B
:1001B0000139F021051405100513080086150130DA
:1001C0008A002608DE21A900290CF000700C0139F4
:1001D000AB00290EF000F00C700C0139AC00290CBA
:1001E0000139AD00290EF000700C0139AE0029086C
:1001F0000139AF00290CF000F00C700C0139B0008F
:10020000290E0139B100290D290D0139F0210514FC
:10021000051086110800061601308A002708DE2125
:10022000A900290CF000700C0139AB00290EF00078
:10023000F00C700C0139AC00290C0139AD00290E0D
:10024000F000700C0139AE0029080139AF00290C0B
:10025000F000F00C700C0139B000290E0139B1002A
:10026000290D290D0139F021051405100612080089
:10027000861601308A002808DE21A900290CF0002A
:10028000700C0139AB00290EF000F00C700C013934
:10029000AC00290C0139AD00290EF000700C0139B9
:1002A000AE0029080139AF00290CF000F00C700CE9
:1002B0000139B000290E0139B100290D290D01398C
:1002C000F02105140510861208002308AB0024084D
:1002D000AC007A292A080319B128013A0319DE284B
:1002E000033A03190B29013A03193829073A031D68
:1002F00008006529E830F2000330F300831203138D
:100300002C08F1002B08F0006F207408A500E830DD
:10031000F2000330F3002B08F0002C08F1006F20EE
:100320007008AB007108AC006430F200F3012C08D7
:10033000F1002B08F0006F207408A6006430F20072
:10034000F3012B08F0002C08F1006F207008AB00BF
:100350007108AC000A30F200F3012C08F1002B0800
:10036000F0006F207408A7000A30F200F3012C0897
:10037000F1002B08F0006F207008A80008008B0126
:10038000831603138501C0308600073083129F0057
:1003900085018601831681130B17831210129012A8
:1003A00090119010FF308F00EF308E0010149701E5
:1003B00083160C148B158B17831208008207FC34EC
:1003C0006034DA34F2346634B634BE34E034FE34A9
:1003D000F634EE343E349C347A349E348E34103409
:1003E0008301B20001222B0801222C0801222D08D2
:1003F00001222E0801222F08012230080122310893
:10040000012A8301B300330C031C082A8517092A2B
:0C0410008513851485100800BF210D2AFB
:02400E00503F21
:00000001FF
